:1000000018308A0000280000FF00030E8301A100C1
:100010000A08A0008A010408A2007708A300780853
:10002000A4007908A5007A08A6007B08A70083131E
:1000300083128C308400801E1F288C1A39288B1E56
:1000400023280B193628220884002308F7002408E7
:10005000F8002508F9002608FA002708FB00200808
:100060008A00210E8300FF0E7F0E09008A110A12FA
:10007000B42A8A110A12BE2A0A108A100A118207AB
:1000800028340C34013406340A108A100A1182070D
:100090000A3400340E3411341F3411341134003456
:1000A000043400340E3411341F341134113400344C
:1000B000043400340E3401340F3411340F3400345E
:1000C00004340E3415340434043404340434003459
:1000D000043404340434043415340E340434003449
:1000E0000034003400340034003400340034003470
:1000F0000034003400340034003400340034003460
:10010000003400340034003400340034003400344F
:100110000A108A100A118F3E03188A0A820041349D
:1001200001342F344234013406344334013447342B
:100130004434013430344534013409344634013414
:10014000423447340234323448340234343449348B
:10015000023436344A34023438344D34E234003414
:100160004E34E23402344F34E23404345034E23456
:1001700006345134E23408345234E2340A3453340D
:10018000E2340C345434E2340E34583401344E34F6
:10019000593401344F345A34013450344B34E1343F
:1001A00010344C34013453345534E2342034313477
:1001B000E13415343234E13416343334E234173454
:1001C0003434E13419343534E234223436340234F0
:1001D00051343734E2341A343834E2341C3439348C
:1001E000E2341E346134023444346234E134253460
:1001F0006334E13424346434E23426346534013425
:1002000007346634013449346734E13428346834BF
:10021000E23429346934E2342B346A3402346234EF
:100220000A148A100A1182070034003400340034A2
:1002300000340034013400341C34E234003400341F
:10024000443404343C3400342834F1340034003471
:1002500001340034013400341534E1340A340034FC
:1002600063340034013400341634E1340134003492
:100270005A3400340134003416340234013400346A
:1002800001340034013400340A148A100A11820740
:100290000C34463465346C343A3420345034613490
:1002A0006E346E346C34753463346B3461342F3493
:1002B0000A34D63476346534723468346534743430
:1002C00074346E3469346E34673400340A148A101E
:1002D0000A1182070C34543469346D346534723435
:1002E00000340A148A100A1182070C34463465342B
:1002F0006C343A342034503465346C346C346534A6
:10030000743473340A3473346C3475347434003494
:100310000A148A100A1182070C34463465346C348E
:100320003A34203449346E34673465346E342034C2
:100330004C34E534673461340A34643465347434DD
:1003400065346B347434653472346134643400342D
:100350000A148A100A1182070C34463465346C344E
:100360003A342034D63476346534723454346534B7
:100370006D34703400340A148A100A1182070C3468
:10038000463465346C343A345234F6346B340034C9
:100390000A148A100A1182070C34463465346C340E
:1003A0003A344D34613474346E3469346E346734A5
:1003B0002034E43472340A347034E53420344D345B
:1003C00069346E347634E434723464346534003421
:1003D0000A148A100A1182070C34463465346C34CE
:1003E0003A3420344F346B34E4346E347434203473
:1003F000663465346C342E3400340A108A140A11C1
:1004000082070C344434723469346634743474347E
:1004100069346434203425346C3475343A342534EA
:1004200030343234753420340A344D346134743409
:100430006E3469346E3467342034253464342034A7
:100440002534253420342534633400340A108A14CA
:100450000A11820753347034613472346134723457
:1004600020347634E43472346434653400340A1051
:100470008A140A1182070C34543469346D3465349B
:10048000723474346934643400340A108A140A11E2
:100490008207743469346D34203400340A108A14AD
:1004A0000A1182070C34543469346D346534723463
:1004B0002034283431343D34533474346F34703440
:1004C0007034293400340A108A140A1182070C345B
:1004D0004D346134783420346D34613474346E3486
:1004E00069346E34673400340A108A140A118207A2
:1004F0000C344D3469346E3420346D3461347434CA
:100500006E3469346E34673400340A108A140A1168
:1005100082070C34543465346D347034653472346D
:1005200061347434753472340A3425346C34643470
:10053000203425346334433400340A108A140A11F9
:100540008207503465346C34323431345F3456347D
:10055000653472345F3432342E34303436340A34F5
:100560005334773465340034B10BB92A3C1401306C
:10057000B100BD170B118A110A122328180883161F
:10058000DF005F080339003A0319D72A83121A08DB
:100590008316DF0083121A088316DF0083121A08FD
:1005A0008316DF00831218121816EE2A83161030F5
:1005B00083126507F800640878020F39F6007608A0
:1005C000F80078080E3C031CEE2A663065078400AC
:1005D0001A088000013065070F39E5008C128A1176
:1005E0000A122328D630840000080319062B013094
:1005F000F800F701F70BFA2AF80BF92A4A30F7004E
:10060000F70B002B00000000800BF72A0034831644
:100610005D0EF039F7000F3083120805770488006B
:100620000000081400000000081000348810F030AA
:1006300083168800831208150000081400000808BB
:10064000080E0F398316DD0083120810000008140D
:1006500000000808080E0F398316DC00831208100A
:100660000030831688005D0EF700F030F70577083C
:100670005C04F8007808DC00DC1F402B8312172B89
:100680005A18452B8312881083165A1C4A2B831242
:1006900088148316000083120811000008108316C6
:1006A0005B0EDC000F30DC055C08DD0083120723E5
:1006B00083165B080F39DC00DD008312072300344A
:1006C00000308316880083128810081108100F303C
:1006D0008316D6008312F22201308316C30043082A
:1006E000033C031C7F2B0330DD00831207230530FE
:1006F0008316D6008312F2228316C30A6F2B0230B0
:10070000DD00831207238316C3014308033C031C47
:10071000962B430883123C208316C400DA01440858
:10072000DB00831216238316C30A852B0530D600FF
:100730008312F2228316C30143083F3C031CB72BEC
:1007400040304307C400DA014408DB00831216235B
:1007500083164308831244208316C4000130DA0054
:100760004408DB00831216238316C30A9C2B8312D2
:100770008A150A168D2883165508831203178D00D3
:1007800083168C130C1483120C080313A900290878
:10079000F800003483165308831203178D00831664
:1007A00003135408831203178C0083168C130C1543
:1007B000831203130B138B138B1BDB2B5530831608
:1007C00003178D00AA308D008C14C03083120313E0
:1007D0008B04831603170C11831203130D1AF32BCA
:1007E00083160317EC2B0D12003483164E08D3002A
:1007F0004F08D4008312CA23013083164E07D1005C
:10080000D03084000008D2005108D3005208D40030
:100810008312CA23003483165008D5008312BB23E9
:100820008316D2017808D100D230D30001305007AE
:10083000D400D5008312BB238316530884007808A4
:1008400080005108F8005208F900831200343D1F5F
:10085000882C3D130330D5009330D4004E08053C5E
:100860000318882C4E08073C031C882C6008610480
:100870000319432C60080319E103E00B432CE10842
:10088000031D432CD7141A308316D00083120B2477
:1008900079088316C6007808C50001304507831221
:1008A000DE00831646088312DF000318DF0A1A30C1
:1008B0008316CE0083125F088316D00083125E0871
:1008C0008316CF008312F5231C308316D0008312C9
:1008D0000B2479088316C4007808C3004308440435
:1008E0000319862C440883125F02031C842C031D09
:1008F000812C5E0883164302031C802C8312842CF7
:100900008312C9148430C600882C83168312C91040
:100910000034BD1D8F2C3D1D8F2C2F14902C2F10BB
:10092000E830831689008312091483168900831224
:100930000910831689008312091430089300831666
:100940001418A42C83129F2C83121308C700E830BC
:1009500083168900831209102F0893008316141838
:10096000B32C8312AE2CE8308900831289148316CD
:100970008900831289100608F038BF0040083F0242
:100980000319C72C40083F06C1063F08C0000034C9
:10099000AF11B010BD110E308316D00083120B249E
:1009A0007908B9007808B8000230B500AE30B4005C
:1009B000B301B20190308316870083120715093006
:1009C000CE00D30100348316560858068039DA0069
:1009D000D61FEF2CD509D609D50A0319D60AD81F78
:1009E000F62CD709D809D70A0319D80AF801F90152
:1009F000F701FA015808031D002D570803191A2D95
:100A00001030D9000310D50DD60DF70DFA0D58088A
:100A10007A02031D0D2D57087702031C162D570867
:100A2000F702031CFA035808FA020314F80DF90D33
:100A3000D90B022D0000DA1F222DF809F909F80A56
:100A40000319F90A8312003410308316D800F70115
:100A5000FA01D50CD40C031C332D5608F7070318E4
:100A6000FA0A5708FA07FA0CF70CF90CF80CD80B2D
:100A7000292D83120034F801F901F701FA018316D8
:100A80005608031D462D55080319602D1030D70058
:100A90000310D30DD40DF70DFA0D56087A02031D7D
:100AA000532D55087702031C5C2D5508F702031CD3
:100AB000FA035608FA020314F80DF90DD70B482D66
:100AC00000008312003420308316D00083120B24E0
:100AD00079088316C9007808C8001530D50083123C
:100AE000BB2378088316CA001630D5008312BB23B7
:100AF00078088316CB002430D5008312BB237808F6
:100B00008316CC002530D5008312BB2378088316CA
:100B1000CD002630D00083120B2479088316CF0035
:100B20007808CE0032304802F7004908FA00003059
:100B3000031C0130FA027708F8007A088312450294
:100B4000031CB02E031DA82D440878020318B02EF4
:100B5000440883164802F7004908FA008312450842
:100B6000031C450FFA0277088316C6007A08C700EF
:100B70004708FA004608C71FC62D4608003CF70084
:100B8000FA014708031C470FFA027708D0007A08D9
:100B9000D100D11BD22DD108031D962E5008FE3C4A
:100BA000031C962E4708FA004608C71FE02D46088A
:100BB000003CF700FA014708031C470FFA027708C8
:100BC000D0007A08D100D11BEC2DD108031D182EBE
:100BD0005008273C031C182E46088312E20703180E
:100BE000E30A831647088312E307E31B062E630814
:100BF0002D3C0318062EFF3A031D022E6208E03C2E
:100C00000318062E2E30E300E030E200E31F162E1C
:100C10006308D13C031C162E031D122E62081F3CD4
:100C2000031C162ED130E3002030E2001B2E831669
:100C30008312E301E20163088316D600831262087F
:100C40008316D5004F08D8004E08D7008312E3243E
:100C500078088316C6070318C70A7908C707FA0178
:100C60004C08D0007A08D1004708D5004608D400C7
:100C70005108D7004C08D600831224257908831622
:100C8000D2007808D100FA014D08D3007A08D400C8
:100C90005208D6005108D5005408D8004D08D70096
:100CA0008312E32479088316C7007808C600460833
:100CB000323CC6004708031C470F602E0030612EEF
:100CC000003CC700FA014A08F800FA1F6A2EC71F45
:100CD000762E6C2EC71B7C2E7A084702031C7C2EB6
:100CE000031D762E4608780203187C2EFA014A0866
:100CF000C6007A08C700952EFA014B08F800C71FF6
:100D0000842EFA1F902E862EFA1B952E47087A0203
:100D1000031C952E031D902E780846020318952E6D
:100D2000FA014B08C6007A08C700AE2EC71BA52ED5
:100D3000C708031D9F2E4608003C0318A52EFA0184
:100D40004B08C6007A08C700AA2EFA014A08C60056
:100D50007A08C7008312E301E2018316BA2E8312D8
:100D6000FA0183164B08C6007A08C7008312E30114
:100D7000E201831646088312D30022308316D00086
:100D800083120B2479088316C5007808C4008312E7
:100D90003D1CF42E19308316D5008312BB23831615
:100DA000D1017808D000FA01831253088316D200CB
:100DB0007A08D3005108D5005008D4005308D70052
:100DC0005208D6008312242579088316D2007808A9
:100DD000D1005208D4005108D300D6016430D500A8
:100DE00083123B257808D300FA0153088316D000FC
:100DF0007A08D1004508D5004408D4005108D7002E
:100E00005008D6008312242579088316D20078086A
:100E1000D1005208D4005108D300D6016430D50067
:100E200083123B257908D2007808D100003483165C
:100E30005508F80154020318202F5408F7002C2FEE
:100E4000F7010830D600D40DF70D550877020318C6
:100E5000F700F80DD60B232F831200348316570B9F
:100E6000322F352F4030D800362FD80101305602AE
:100E7000D80758088038D900DA015908DB008312F6
:100E800016230034831655080C3A83120319612F78
:100E9000063A03196D2F023A0319752FEC3A03191C
:100EA0007C2F013A0319842F133A03198C2F323AFD
:100EB0000319942F013A03199B2F133A0319A22FF8
:100EC000AA2F8316DA010130DB00831216230230C9
:100ED0008316D6008312F222B22F01308316D60079
:100EE0000230D70083122E27B22F8316DA0110307A
:100EF000DB0083121623B22F01308316DA00E130B3
:100F0000DB0083121623B22F01308316DA00023081
:100F1000DB0083121623B22F01308316DA00EF3084
:100F2000DB0083121623B22F01308316DA00DB01B7
:100F300083121623B22F01308316DA00DB008312EE
:100F40001623B22F01308316DA00EF30DB00831254
:100F50001623B22F01308316DA005508DB00831206
:100F60001623B22F0034780883164D08D40064305D
:100F7000D5008312172777088316CD007808303004
:100F8000031DC92FCE1CD22FCE19D22F4E1A2030BE
:100F9000CC2FCE114E124E14F8077808D5008312CC
:100FA000422783164D08D4000A30D5008312172734
:100FB00077088316CD0078083030031DE52FCE1951
:100FC000EB2F4E1CEB2F4E1A2030F8077808D50077
:100FD0008312422783163030CD074D08D500831287
:100FE00042278A150A12202C0C1EF42F83164C0857
:060FF00083129900003499
:1010000004088316D4004E0EF038D000D007E23E1C
:10101000D100323ED3004E080F39D107D107D30794
:10102000E93ED200D207D2074D0E0F39D207D307BF
:10103000D20DD30DD309D30D4D080F39D307D00DE1
:101040000730CF000A30D307D203031C2328D2076E
:10105000D103031C2728D107D003031C2B28D0075A
:10106000CF03031C2F28CF308400073054055413BE
:101070008407D3300402031954170008F700031D36
:101080004928541B4928541A5928D4194928203072
:101090004C28D41554123030F707CE010408CD0087
:1010A0007708D5008A11831242278A1583164D08C6
:1010B0008400840A541F392883128A150A12112CBD
:1010C000203083164F1E3030D0004E08F700CE1F60
:1010D0007028F709F70A7708CE002D30D000CF1717
:1010E0004E08D4006430D5008A11831217278A1560
:1010F00077088316CE0030307807D1004E08D40030
:101100000A30D5008A11831217278A1530307707E5
:101110008316D30030307807D2005008F700CF1D77
:101120009328CF1F4F114F1AA028CF1FBB284F194C
:10113000BB287708D100CF18BB287708D200BB287E
:1011400030305102031DBB287708D1002030D00079
:10115000CF1DAE284F11CF14CF1FCF103030520209
:10116000031DBB287708D2002030D100CF1DAE2848
:10117000CF10CF1F4F104F1DC4285008D5008A1123
:10118000831242278A158316CF1CCD285108D5001B
:101190008A11831242278A1583164F1CD6285208BB
:1011A000D5008A11831242278A1583165308D50069
:1011B0008A11831242278A158A150A123E2CF701DA
:1011C000F80183164C0803104D18F707F70CF80CBC
:1011D000CD18F707F70CF80C4D19F707F70CF80CBA
:1011E000CD19F707F70CF80C4D1AF707F70CF80CA8
:1011F000CD1AF707F70CF80C4D1BF707F70CF80C96
:10120000CD1BF707F70CF80C831200340408831683
:10121000D100CB1F1329D117511ED10ACA09CB09FE
:10122000CA0A0319CB0A4B0EF038CD00CD07E23EB7
:10123000CE00323ED0004B080F39CE07CE07D00784
:10124000E93ECF00CF07CF074A0E0F39CF07D007AF
:10125000CF0DD00DD009D00D4A080F39D007CD0DD4
:101260000730CC000A30D007CF03031C3329CF0747
:10127000CE03031C3729CE07CD03031C3B29CD0722
:10128000CC03031C3F29CC30840007305105511397
:1012900084035105031D5329511A840A511A5329F5
:1012A0002030F70070298407D03004020319511749
:1012B0000008F700031D6429511B6429511A7C2979
:1012C000D119642920306F29D11F6C292D30F700E6
:1012D00084035113D1137029D11551123030F707FF
:1012E000CB010408CA007708D5008A11831242276F
:1012F0008A1583164A088400840A511F54298312D0
:101300000034831644080B3C031D91291A30CE008B
:10131000D001CF018A118312F5238A15DF01DE0186
:1013200083164408083C031DA12A01308312480794
:101330008316CA00D4000630D5008A1183121727FD
:101340008A1577088316C600460DF700F70DF70DCE
:10135000F830F7057708013E8A11831210218A15AB
:10136000F8008316C7004708DF3C0318A12A460D82
:10137000F700F70DF70DF830F7057708043ECA00BF
:101380004A0A8A11831210218A15FA0083164A0824
:101390008A11831210218A15DA007A08DB0083167D
:1013A000460DF700F70DF70DF830F7057708023E08
:1013B000CA004A0A8A11831210218A15FA0083167C
:1013C0004A088A11831210218A15DC007A08DD0090
:1013D0008316460DF700F70DF70DF830F70577087F
:1013E0008A11831210218A15F8008316C800470855
:1013F000E13C031D272A4808D5008A118312BB232C
:101400008A1578088316C900460DF700F70DF70D09
:10141000F830F7057708063ECB004B0A8A11831295
:1014200010218A15FA0083164B088A1183121021A5
:101430008A158316CC004908D4004C08D5008A11BF
:10144000831217278A15D9017808D8008316470810
:10145000E23C031D602A4808D0008A1183120B2445
:101460008A1579088316CA007808C900460DF70066
:10147000F70DF70DF830F7057708063ECC004C0A5B
:101480008A11831210218A15FA0083164C088A11DA
:10149000831210218A158316CD007A08CE004A08DF
:1014A000D4004908D3004E08D6004D08D5008A1153
:1014B00083123B258A157908D9007808D80083164D
:1014C0004708EF3C03187F2A4808D5008A11831289
:1014D000BB238A1578088316C90047080739F80026
:1014E0004908F700F8080319792A0310F70CF80BDC
:1014F000752A770801398312D800D901831683121F
:101500005B085902031C8E2A031D8A2A58085A02B6
:1015100003188E2A5B08D9005A08D80059085D02C2
:10152000031C9C2A031D982A5C08580203189C2A55
:101530005D08D9005C08D8005714BB019830BA0088
:10154000831644080A3C031DD32A8312C908031DCD
:10155000AB2A8316D32A0130F7004A08F800031992
:10156000B52A0310F70DF80BB12A7708FF3AC90521
:10157000BB010230BA004A08FB3E0318D22A053EDE
:10158000802ED22A1A308316CE00D001CF018A11C4
:101590008312F5238A15DF01DE01D22AC201D22A85
:1015A0003D12D22A83164408453C031D5F2C83124A
:1015B00057104E080B3C031DE72A49084B05003A1B
:1015C000031DE72ACE01BC133C13D001CF01C9088B
:1015D0000319C22B8316C5014508073C031CC02B09
:1015E0008312CA0A0730CA054908F7004A08F800FA
:1015F0000319FE2A0310F70CF80BFA2A771CBD2BEF
:101600004A08F83E0318B62B083E892E8316C901F6
:1016100049088A11831244218A158316C90AF700E2
:10162000D5008A11831242278A151D30831649027C
:10163000031D082B8312B62B8316C90149088A1192
:10164000831266218A158316C90AF700D5008A110C
:10165000831242278A15063083164902031D1E2B6A
:101660008312B62B8316C90149088A11831271218E
:101670008A158316C90AF700D5008A1183124227FA
:101680008A15123083164902031D342B8312B62BA0
:101690008316C90149088A11831288218A15831685
:1016A000C90AF700D5008A11831242278A151B3018
:1016B00083164902031D4A2B8312B62B8316C901D8
:1016C00049088A118312A8218A158316C90AF700CE
:1016D000D5008A11831242278A150E3083164902DB
:1016E000031D602B8312B62B8316C90149088A118A
:1016F0008312BB218A158316C90AF700D5008A1107
:10170000831242278A15083083164902031D762B5F
:101710008312B62B8316C90149088A118312C82186
:101720008A158316C90AF700D5008A118312422749
:101730008A151B3083164902031D8C2B8312B62B8E
:101740008316C90149088A118312E8218A15831674
:10175000C90AF700D5008A11831242278A15103072
:1017600083164902031DA22B8312B62BC801BB01AD
:101770002D30BA008316C02B83128316C50AEC2ABB
:101780005F2C83123F08F93C031DD12B1A308316BE
:10179000CE00D001CF018A118312F5238A15DF0113
:1017A000DE015F088316D40083125E088316D3001F
:1017B000D6013C30D5008A1183123B258A15790861
:1017C0008316CA007808C90083125F088316D40004
:1017D00083125E088316D300D6013C30D5008A11EF
:1017E00083123B258A1577088316CB00CC014C0861
:1017F0008A118312FD218A158316CC0AF700D500C1
:101800008A11831242278A150A3083164C02031D5F
:10181000F72B103084004A08CE004908CD0083120F
:1018200000283A308316D5008A11831242278A1580
:1018300083164B08CD000130CE008A118312B32FDE
:101840008A1512308316CD004D088A118312FD21AE
:101850008A158316CD0AF700D5008A118312422714
:101860008A151C3083164D02031D242C8312530845
:101870008316CE001F30CF008312602820308316DD
:10188000D5008A11831242278A1525308316D50088
:101890008A11831242278A1520308316D5008A11B7
:1018A000831242278A154D088316D5008A118312A8
:1018B00042278A15C801BB010F30BA0083164408BD
:1018C000093C031D562D83125718682C8316562D7C
:1018D0005710480DF700F70DF70DF830F7057708AA
:1018E000013E8A1110218A15F8008316C700831261
:1018F000480DF700F70DF70DF830F70577088A1156
:1019000010218A15F8008316C8004708E13C031D22
:10191000B62C8312480DF700F70DF70DF830F705D8
:101920007708063E8316CA004A0A8A1183121021DC
:101930008A15FA0083164A088A11831210218A1523
:101940008316CB00831258088316CC004B08CD00B9
:101950008312DF2078088316CC004808D3004C0897
:10196000D4008A118312CA238A1583164708E23CE1
:10197000031DF52C8312480DF700F70DF70DF83015
:10198000F7057708063E8316CA004A0A8A118312B1
:1019900010218A15FA0083164A088A118312102131
:1019A0008A158316CB007A08CC0083125908831657
:1019B000D500831258088316D4004C08D7004B0872
:1019C000D6008A11831224258A1579088316CD0042
:1019D0007808CC004808CE004D08D0004C08CF0055
:1019E0008A118312F5238A1583164708EF3C0318E2
:1019F000322D4808D5008A118312BB238A15780836
:101A00008316C5008312D8080319182D83164708BA
:101A10000739C9000130F7004908F8000319142DEF
:101A20000310F70DF80B102D7708C504292D83122C
:101A3000831647080739C9000130F7004908F80044
:101A40000319262D0310F70DF80B222D7708FF3A06
:101A5000C5054808D3004508D4008A118312CA235B
:101A60008A1583168312C80101308316D60002300E
:101A7000D7008A1183122E278A158316C9014908B7
:101A80008A11831226228A158316C90AF700D50007
:101A90008A11831242278A150C3083164902031DCE
:101AA0003F2D8312BB010F30BA0083168312480802
:101AB000FA3E03187D2E063E952E83164408083AFA
:101AC0008312031D972D8316C90149088A118312B9
:101AD00037228A158316C90AF700D5008A118312A6
:101AE00042278A15093083164902031D652D0A30E5
:101AF000D6000230D7008A1183122E278A1583164A
:101B0000C90149088A11831245228A158316C90A18
:101B1000F700D5008A11831242278A1504308316F4
:101B20004902031D812D01308312C800972D7D2E9F
:101B300083164408083A8312031DB62D8316C90183
:101B400049088A1183124E228A158316C90AF700A2
:101B5000D5008A11831242278A1510308316490254
:101B6000031DA02D02308312C800B62D7D2E8316D2
:101B70004408083A8312031DF32D8316C90149084E
:101B80008A11831263228A158316C90AF700D500C9
:101B90008A11831242278A150C3083164902031DCD
:101BA000BF2D03308312C8000A308316D6000230DE
:101BB000D7008A1183122E278A1525308316D50067
:101BC0008A11831242278A1520308316D5008A1184
:101BD000831242278A1520308316D5008A1183127A
:101BE00042278A15F32D7D2E83164408083A831266
:101BF000031D302E8316C90149088A1183127422ED
:101C00008A158316C90AF700D5008A118312422764
:101C10008A150C3083164902031DFC2D04308312F3
:101C2000C8000A308316D6000230D7008A1183120A
:101C30002E278A1525308316D5008A118312422754
:101C40008A1520308316D5008A11831242278A15FF
:101C500020308316D5008A11831242278A15302E30
:101C60007D2E83164408083A8312031D6F2E05301B
:101C7000C8008316C90149088A11831285228A1572
:101C80008316C90AF700D5008A11831242278A15E4
:101C90000C3083164902031D3B2E10308400831242
:101CA00045088316CB00831244088316CA008312AA
:101CB000062120308316D5008A11831242278A1507
:101CC000DF308316D5008A11831242278A154330EC
:101CD0008316D5008A11831242278A156F2E7D2E16
:101CE00083164408083A8312031D7C2EC80157103E
:101CF000BB010230BA007C2E7D2E8A110A16FA2A08
:101D00000A108A140A158207C12AC22ACF2ACE2AAB
:101D1000D02A0A108A140A158207062B1C2B322B94
:101D2000482B5E2B742B8A2BA02B0A108A140A15C1
:101D300082075D2D982DB72DF42D312E702E831630
:101D40004408CC008A118312F4278A15003420300D
:101D50008316C40083129F2656308316C400831254
:101D60009F268316C30143088A1183129D228A1578
:101D70008316C30AF700C40083129F26123083160D
:101D80004302031DB32E0D30C40083129F2600347E
:101D90003D15320833040319D52E32080319B30355
:101DA000B20BD52EB3080319BC143408350403193B
:101DB000E12E34080319B503B40BE12EB50803195D
:101DC0003C15360837040319ED2E36080319B703FE
:101DD000B60BED2EB7080319BC15380839040319E2
:101DE000F92E38080319B903B80BF92EB9080319ED
:101DF0003C163A083B040319052F3A080319BB03A4
:101E0000BA0B052FBB080319BC1654085504031957
:101E1000112F54080319D503D40B112FD50803191A
:101E20003D17D6080319152FD6038A150A163D2A21
:101E30006630640784000008FC0083168C120130B1
:101E4000831264070F39E40083168C167C08F800AF
:101E500083128A150A16442A83164508393C031C46
:101E6000362F30304502F8003B2F3B2F4508DF3935
:101E7000C93EF8003B2F831200348316CB1B542F2E
:101E80000F30F7004A0EF7050A30770203184B2F80
:101E90003030F7074D2F4B08F7077708CC008A1131
:101EA0008312F4278A1583160F30CA050A304A02B6
:101EB00003185C2F30305E2FCB134B08CA074A083B
:101EC000CC008A118312F4278A1500348316C908BE
:101ED000031D742F4608AB004708AC004808AD004E
:101EE0008312D716A02F8316C9080319A12F8312B6
:101EF000D71A7C2F8316A12F20308316CC008A118D
:101F00008312F4278A1583162B08CC008A118312BA
:101F1000F4278A1583162C08CA003730CB008312A9
:101F20003D2783162D08CA003730CB0083123D278A
:101F30000D308316CC008A118312F4278A15D7122C
:101F4000831683120034831606168312061EC52FCD
:101F50005719C32F57158316861600308312861A19
:101F60000130003A031DC22F59085B02031CC12F28
:101F7000031DBE2F5A0858020318C12FD80A03198F
:101F8000D90AC22FC42FE12FE12F571DE02F57117F
:101F90008316861600308312861A0130013C03191D
:101FA000DF2F5D085902031CDF2F031DDB2F5808AC
:101FB0005C020318DF2F58080319D903D803E12F57
:101FC000E12F8316200883125802031DED2F83167C
:101FD0002108831259020319F22F571CF22FBB015B
:101FE0009830BA0059088316A10083125808831646
:0A1FF000A00083128A150A16F82BD0
:102000008316430F19288312B301B201B501B4013D
:10201000B701B601B901B801BC103C11BC113C12AA
:10202000BC133C13BD10CE01D001CF01CC01162B47
:10203000831683124C08003A03192228013A031927
:1020400031284728491483164308853C031D2F284F
:1020500001308312CC004910CE01D30183168312C4
:10206000472883164308053C031D45288312CC01ED
:102070000B30CE00AF01B001903083168700831281
:102080000711BD114914D301831683124728500844
:10209000003A03194F28013A03195A286228831677
:1020A0004308813C031D582801308312D000831659
:1020B000831262288316430B60288312D001831693
:1020C000831262284F08003A03196A28013A03195B
:1020D00075287F2883164308023C031D73280130AE
:1020E0008312CF00831683127F2883164308823C15
:1020F000031D7D288312CF01831683127F284E088B
:10210000F13E0318F32A0F3E172B4B084905003AFE
:1021100003198D280B30CE00F32A4F0BB0284C0B3F
:10212000B028BD1EB0288316D0010A1283120B24DA
:102130000A167908B3007808B200AF15AF16AF14CD
:10214000AF172F152F162B308316D0000A128312CB
:102150000B240A167908E1007808E0000130CE006F
:10216000F32A83164308413A83120319BB28C33A62
:102170000319D228D728AF11AF12B01490308316AC
:10218000870083120715BD150A308316D0000A1286
:1021900083120B240A167908B5007808B4000230BF
:1021A000CE00D7280A12C8240A16AF12D728F32A5D
:1021B000500BE8281E308316D0000A1283120B241D
:1021C0000A167908B5007808B4000330CE00F32A67
:1021D00083164308423A83120319F228C03A0319BE
:1021E0000A290F29BD11B010AF1190308316870056
:1021F00083120711AF120C308316D0000A1283121B
:102200000B240A167908B3007808B200C20A083015
:10221000CE000F290A12C8240A16AF120F29F32A7A
:1022200083164308423A831203191A29C03A031944
:102230003229362990308316870083120715B01093
:10224000BD1104308316D0000A1283120B240A1623
:102250007908B5007808B40004308316AA00831208
:10226000CE0036290A12C8240A163629F32A831604
:102270004308423A831203194129C03A03196029DD
:102280006529AF168316AA0B53290630D0000A120F
:1022900083120B240A167908B5007808B4000530BB
:1022A000CE00652983160230D0000A1283120B2457
:1022B0000A167908B5007808B4000C30CE006529FC
:1022C0000A12C8240A16AF126529F32A8316430896
:1022D000423A831203197029C03A03197F298429CD
:1022E000AF1208308316D0000A1283120B240A168C
:1022F0007908B5007808B4000430CE0084290A12A9
:10230000C8240A16AF128429F32A83164308423AD6
:10231000831203198F29C03A031999299D29AF11F6
:10232000AF12B301E430B200B014BD150E30CE00D0
:102330009D290A12C8240A169D29F32A83164308E8
:10234000423A83120319B129013A0319B429C73A51
:102350000319D529063A0319D629833A0319DA292C
:10236000F1293D10C201F129AF110A1263250A16A5
:1023700022308316D0000A1283120B240A16790821
:102380008316C5007808C4008312510883164402DE
:102390008312B600831645088312B7005208031C47
:1023A000520FB7020730CE00F129F1290A12C824D2
:1023B0000A16F129D301AF119030831687008312DA
:1023C0000711AF120C308316D0000A1283120B24AF
:1023D0000A167908B3007808B200C20A0830CE00A5
:1023E000F129F32A83164308423A83120319052A76
:1023F000013A0319082AC73A0319102A063A0319A1
:10240000112A833A0319152A2C2A3D10C2012C2ABD
:10241000AF155208B7005108B6000630CE002C2A7E
:102420002C2A0A12C8240A162C2AD301AF11903084
:102430008316870083120711AF120C308316D00069
:102440000A1283120B240A167908B3007808B20026
:10245000C20A0830CE002C2AF32A83164308413AD8
:102460008312031D522A4F0B4A2A10308316D500BF
:102470000A128312BB230A167808420203184A2A5A
:10248000BD1E4A2AAF16AF15B5019830B4000A3008
:10249000CE00512AC915AF10AF132F112F120B30D8
:1024A000CE00522AF32A83164308413A83120319B5
:1024B000602A033A0319662A063A0319702A812A08
:1024C00090308316870083120715812A9030831677
:1024D0008700831207110A30B300BA30B200812A94
:1024E000AF1290308316870083120711AF10AF131D
:1024F0002F112F122F17B5015B30B4000D30CE0015
:10250000812AF32A83164308423A8312031D9F2A25
:102510000A308316D0000A1283120B240A16790897
:10252000B5007808B400AF11AF12B014BD159030EB
:1025300083168700831207150230CE009F2AF32AE4
:10254000831643080A3A8312031DA72AA72AF32AEF
:1025500083164308423A8312031DB12A2F13CE017A
:10256000B12AF32A83164308413A83120319BC2A7D
:10257000C33A0319EE2AF22AB010BD11500BD82A23
:10258000AF15AF163D1417308316D0000A12831210
:102590000B240A167908B5007808B4000A126325DE
:1025A0000A165208B7005108B6000630CE00ED2AD0
:1025B000AF1190308316870083120711AF120C30D1
:1025C0008316D0000A1283120B240A167908B3006E
:1025D0007808B200C20A0830CE00F22A0A12C824D3
:1025E0000A16F22AF32A83164308C4000A128A152F
:1025F000831281290A168A11C90803190B2B9030FE
:1026000083168700831287143014E83083168900FC
:1026100083120915162B90308316870083128710BA
:102620003010E830831689008312091100340A142F
:102630008A140A1182078528B128D8281029372939
:1026400085299E29F2292D2A532A822AA02A662921
:10265000A82AB22A571E922B831628080F3C03186B
:10266000772BA801270CC600260CC500C60CC50C8C
:10267000C60CC50CC60CC50CC60CC50C0730C6056F
:1026800045088312C4000230831646078312C50032
:102690004508023C031C542B031D522B44081B3CD1
:1026A000031C542BBD16552BBD124E08093C0319B3
:1026B000732B4E080D3C0319732BCE080319732B93
:1026C00029308316D0000A1283120B240A167908C7
:1026D000FA007A084502031C732B031D722B440871
:1026E0007802031C49168316A701A601892B8312C1
:1026F0001F151F19792B1E08FA0083161E08C30028
:102700007A08C4004308A6070318A70A4408A707C5
:10271000A80A0830F80083121F08C73978049F0000
:102720005712A02B1F151F19932B83161E088312F7
:10273000C3000030F8001F08C73978049F005716FF
:102740008A150A160B2C47088316A500A509283000
:10275000D5000A128312BB230A167808CB00BC1CD2
:10276000B52BBC104130F800D02C3C1DBB2B3C11CC
:102770004230F800D02CBC1DC12BBC114330F800F6
:10278000D02C3C1EC72B3C124430F800D02CBC1E71
:10279000CD2BBC124530F800D02CBD1CDA2B831693
:1027A000A51BD82B8312BD100530F800D02C831642
:1027B000E32B83128316A51FE32B8312BD148530F0
:1027C000F800D02C83168312471CE92B4230CD0031
:1027D000EB2B2030CD00BC1FFD2B47080139003A00
:1027E000031DFA2BD608031DF92BBC130130F8008A
:1027F000D02CFC2BE430D600052C471C052CE430F3
:10280000D600BC178130F800D02CD71C0C2CD71068
:102810003C138230F800D02C3C1F1B2C8316A51CC7
:10282000132CA519192C83123C138230F800D02CDC
:102830008316282C83128316A51C282C251D282CD2
:10284000A51D282C83123C170230F800D02C8316CB
:102850008312C6080319362C46088316A500831276
:10286000C60183162508F8008312D02C8316251E76
:10287000492C831249080439003A031D462C4B1D8C
:10288000462C3C1349158230F800D02C49154B2CAE
:102890008316831249118316A51E5D2C83124908E5
:1028A0002039003A031D5B2CCB1E5B2C3C13C91650
:1028B0008230F800D02CC916831683123D1A692C79
:1028C000491E692C4B1E692C3C133D168230F800C2
:1028D000D02C41083F05003A03199B2C8316A30115
:1028E0002308073C031C9A2C0130A4002308F8009D
:1028F00003197E2C0310A40DF80B7A2C83124108C7
:102900003F0583162405003A0319982C2408FF3A42
:102910008312C1058316220EF700F030F705770801
:10292000803E2307013E073EF8008312D02C831619
:10293000A30A702C83123F08FF3A4105003A03199D
:10294000CE2C8316A3012308073C031CCD2C013099
:10295000A4002308F8000319B12C0310A40DF80BF0
:10296000AD2C83123F08FF3A410583162405003A37
:102970000319CB2C2408FF3A8312C1058316220EBB
:10298000F700F030F70577082307013E073EF8000F
:102990008312D02C8316A30AA32C83120030F800D4
:0629A0008A150A16102C36
:103000001F3083055730F700203084008001840A88
:10301000F70B0628F801F901FA01FB01FC01FD019B
:10302000FE015030F700A03084008001840AF70BC5
:103030001528A00184011F30830583161F149F14D7
:103040001F159F110C309900263098009030831284
:103050009800A801A901AA010130AB00AC01AD01A3
:10306000AE01F601FC015711D7118316A001A10191
:10307000A201A301A401A501831257128316A60180
:10308000A701A801A901AA01AB01AC01AD018312FE
:10309000D7128316B2018312D30114308316D600DF
:1030A0000A128A118312F2220A168A153D10C601ED
:1030B0000730F700F71D6428073081018130840054
:1030C0000008C0390F388000640081308400000897
:1030D000C0397704800083161F149F101F159F119D
:1030E00083121F179F1783169F1783121F149412A2
:1030F0009030831687008700870030308312940059
:103100004030831694000030F80083121F08C7393E
:1031100078049F000A128A11602B0A168A15013062
:103120008316D5000A128A118312BB230A168A1548
:10313000780FC9298316CE010230D0001630CF0097
:103140000A128A118312F5230A168A1564000230C6
:103150008316CE00D0011E30CF000A128A118312CE
:10316000F5230A168A15640004308316CE00D001B8
:10317000E430CF000A128A118312F5230A168A1549
:10318000640006308316CE000130D0003130CF000D
:103190000A128A118312F5230A168A1564000A306E
:1031A0008316CE000730D0002730CF000A128A11D4
:1031B0008312F5230A168A15640008308316CE00A0
:1031C0000130D0007D30CF000A128A118312F5231E
:1031D0000A168A1564001E308316CE000230D00015
:1031E0001630CF000A128A118312F5230A168A15A7
:1031F00064000C308316CE000130D0003130CF0097
:103200000A128A118312F5230A168A1564000E30F9
:103210008316CE003530D000A430CF000A128A11B8
:103220008312F5230A168A15640010308316D30022
:103230000430D4000A128A118312CA230A168A158E
:10324000640015308316D3005A30D4000A128A1154
:103250008312CA230A168A15640016308316D30017
:103260001430D4000A128A118312CA230A168A154E
:10327000640017308316CE000630D0008E30CF00A9
:103280000A128A118312F5230A168A15640019306E
:103290008316D3003C30D4000A128A118312CA2349
:1032A0000A168A151A308316CE00D001CF010A12F1
:1032B0008A118312F5230A168A1564001C308316BE
:1032C000CE00D001CF010A128A118312F5230A160B
:1032D0008A1520308316CE000230D000BC30CF00DB
:1032E0000A128A118312F5230A168A1522308316D0
:1032F000CE00D0015B30CF000A128A118312F52371
:103300000A168A1525308316D3000830D4000A1215
:103310008A118312CA230A168A1524308316D30011
:103320000430D4000A128A118312CA230A168A159D
:10333000640026308316CE00D0013230CF000A124E
:103340008A118312F5230A168A1528308316D300B2
:103350003E30D4000A128A118312CA230A168A1533
:1033600029308316CE000330D0005230CF000A122D
:103370008A118312F5230A168A152B308316CE0084
:10338000D001F030CF000A128A118312F5230A16F9
:103390008A15D301FF30BF00C000C101831642105F
:1033A0008312D710C901CA01BD110730BE00033016
:1033B000D5009330D4003D17C9100630CE000A1254
:1033C0008A1127240A168A15CE01C8015710C20196
:1033D000E401E501AF01B00190308316870083124C
:1033E00007110A128A1189240A168A15FF308316DA
:1033F000C3008A11831200208A150A12A7260A1612
:103400008B1683168C16C03083128B048316B3017F
:1034100001308312B1000C308316D5000A128A11D4
:10342000831242270A168A158316C30143080A121B
:103430008A1183129D220A168A158316C30AF70081
:10344000D5000A128A11831242270A168A151230F1
:1034500083164302031D162A8312BC12BB01983047
:10346000BA003D1290308316870083120710640063
:10347000BD1F3E2ABD130A12C82E0A166508640233
:103480000319F42B0A12182F0A1678088316B100B4
:103490003108203C031D4F2A0130B200F52BB20841
:1034A0000319F52B31080D3C031DB62B03303202F6
:1034B000F83E0318B42B083E8312832C8316B42BDA
:1034C0008316B42B83163808C5000A1283122C27E2
:1034D0000A16780E8316C400F030C4053908C500FA
:1034E0000A1283122C270A16780883164407B8009C
:1034F0003A08C5000A1283122C270A16780E831682
:10350000C400F030C4053B08C5000A1283122C2702
:103510000A16780883164407B9003708563C031D7D
:10352000972A0A128312A7260A168316B42B370885
:10353000573C031DA02A38088312C6008316B42BFB
:10354000B50135082A3C031CB22B3508CC000330EA
:10355000CD000A128312DF200A1678080A128A1197
:1035600088200A168A15F8008316BC0037083C022A
:10357000031DB02B3508CC000330CD000A12831296
:10358000DF200A16013078070A128A1188200A16ED
:103590008A15F8008316BD003508CC000330CD0035
:1035A0000A128312DF200A16023078070A128A11E3
:1035B00088200A168A15F8008316BE00BD08031974
:1035C000AF2B3D0BFF2A3608573C031DEF2A32086C
:1035D000053C031DEF2A3E088400380880003E08A1
:1035E00084000008C3003708C600C7014308C800AC
:1035F000C9010A12831266270A16AE2B83163D08EC
:10360000023C031D2A2B3608573C031D142B32089D
:10361000073C031D142B3E0884003908800001304C
:103620003E0784003808800001303E07840000080F
:10363000C3003E0884000008C4003708C6004308E1
:10364000C7004408C800C9010A12831266270A1677
:10365000AE2B83163D08E03C0319AF2B3D08E13C3F
:10366000031D5C2B3608573C031D452B3208053CD7
:10367000031D452B3E08D3003808D4000A128A11D6
:103680008312CA230A168A1583163E08D5000A1229
:103690008A118312BB230A168A1578088316C30081
:1036A0003708C600C7014308C800C9010A128312BF
:1036B00066270A16AE2B83163D08E23C031DA52B98
:1036C0003608573C031D802B3208073C031D802B16
:1036D00001303E07C300D3003808D4000A128A1113
:1036E0008312CA230A168A1583163E08D3003908A6
:1036F000D4000A128A118312CA230A168A15831665
:1037000001303E07C300D5000A128A118312BB2381
:103710000A168A1578088316C4003E08D5000A12D6
:103720008A118312BB230A168A1578088316C500EE
:103730003708C6004408C7004508C800C9010A1276
:10374000831266270A16AE2B83163708C600C701F8
:10375000C801C9010A12831266270A168316B22B02
:10376000B50AA12AB42B8316B201F52B013032021F
:10377000F73E0318F52B093E83128F2C8316310870
:10378000B6000230B200F52B83163108B7000330C3
:10379000B200F52B83163108B8000430B200F52BC7
:1037A00083163108B9000530B200F52B83163108B5
:1037B000BA000630B200F52B83163108BB00073083
:1037C000B200F52B83163108BC000830B200F52B8F
:1037D00083163108BD000930B200F52B831631087D
:1037E000BE000A30B200F52B83160A128312A32FF3
:1037F0000A1683163308FB3E03187B2C053E831202
:103800009C2C3C1C0C2C3C100A128A1189240A1690
:103810008A158A112A2B8A1583167B2C8A11A32BD1
:103820008A1578088316B4003408C3008A118312FD
:1038300000208A158316B40803192B2C421C2B2C4C
:103840005730C600C7013408C800C9010A128312E4
:1038500066270A1683167B2C0A128A1127240A1659
:103860008A1583167B2C571C6C2C480DF700F70D1E
:10387000F70DF830F7057708013E0A128A1110217A
:103880000A168A15DF3C03186C2C01308316D6000B
:103890000230D7000A128A1183122E270A168A15BF
:1038A0001030840059088316CB0083125808831601
:1038B000CA000A12831206210A1604308316C300B6
:1038C0002030D5000A128A11831242270A168A155F
:1038D0008316C30B602C831283167B2C8316C601C0
:1038E000C701C8010130C9000A12831266270A16EF
:1038F00083167B2C8316B30A3308053C0319B301E6
:103900008312372A63000A108A100A158207622A76
:103910005E2A622AB32B622AB32BB32B602A0A10C9
:103920008A100A158207BE2BC42BCA2BD02BD62B8C
:10393000DC2BE22BE82BEE2B0A108A100A158207EB
:0A394000012C0E2C2C2C332C6E2CC5
:02400E00723FFF
:00000001FF
